:020000040000FA
:020000000428D2
:08000800FF30A200FF30A3004D
:1000100002212821A701A801A901A0100F30522117
:100020000F304921A413472124134821A51146214B
:100030000030702100306121A2137C2122137D2128
:10004000A3117921CC20A413A71F2728A417472187
:100050002413A81F2C2824174821A511A91F3128D3
:10006000A51546210E305221F3200F305221CC200D
:10007000A413271F3C28A41747212413281F412815
:1000800024174821A511291F4628A51546210D3002
:100090005221F3200F305221CC20A413A71E512847
:1000A000A41747212413A81E562824174821A51158
:1000B000A91E5B28A51546210B305221F3200F30D5
:1000C0005221CC20A413271E6628A41747212413ED
:1000D000281E6B2824174821A511291E7028A51554
:1000E000462107305221F3200F305221CC20A41397
:1000F000A71D7B28A41747212413A81D8028241797
:100100004821A511A91D8528A51546210E30492194
:10011000F3200F304921CC20A413271D9028A417C9
:1001200047212413281D952824174821A511291D8E
:100130009A28A51546210D304921F3200F30492179
:10014000CC20A413A71CA528A41747212413A81C5E
:10015000AA2824174821A511A91CAF28A5154621B6
:100160000B304921F3200F304921CC20A413271C48
:10017000BA28A41747212413281CBF282417482174
:10018000A511291CC428A515462107304921F320B3
:100190000F3049212228CB2807212A08A600201D3C
:1001A000D328A014D428A010A01CF2282608A70049
:1001B000A010A01CDC28E52807212A08A800201D83
:1001C000E328A014E428A010D928A010A01CE92836
:1001D000F22807212A08A900201DF028A014F128E0
:1001E000A010E62808003230F528AA00F430AB0051
:1001F000FC30AC002A082B07031C00342C07031822
:10020000FE28080003309F0084211F1387299818B7
:10021000152918191F298C1E25298B138B1B0D29B5
:100220001A088B172015AA0008008B138B1B1529A1
:1002300018121A081A081A0818168B1707298B1390
:100240008B1B1F291A088B1707292011080008008B
:1002500023117A21A3147B218421181398161812D4
:1002600018151810181D37290C3099003B2918193A
:100270003B29023099008721981718131816181176
:100280001A081A081A080030990008005B295E292C
:100290005E29AA002A0EF039AB0025080F392B047D
:1002A000A5005B29AA002A080F39AB002408F03901
:1002B0002B04A4005E292508860008002408850078
:1002C0000800AA0023080F39AB002A080F39AD0037
:1002D0000430AE008A21AC002C082B04A3007E2938
:1002E000AA002A080F39AB002208F0392B04A2001B
:1002F00081297E297E297E2981298129230866007A
:100300000800220865000800831603130800831202
:1003100003130800AE002E08003C031C9029962908
:100320000310AD0D01302E02AE008B292D08080000
:02400E00103F61
:00000001FF
